:100000000C942A000C9447000C94380C0C94560164
:100010000C9447000C9447000C9447000C94470044
:100020000C9447000C9447000C9447000C9423094F
:100030000C945F090C9447000C9447000C94470003
:100040000C9447000C9447000C9447000C94470014
:100050000C94470011241FBECFE5D4E0DEBFCDBF16
:1000600010E0A0E6B0E0EAE6FEE102C005900D92E5
:10007000A036B107D9F711E0A0E6B0E001C01D92AB
:10008000A136B107E1F70E9470060C94340F0C946E
:1000900000008C9A8FB583638FBD8EB589608EBD4D
:1000A00019BC18BC08959B01AC01E0EAFFE007C051
:1000B000CF010197F1F721503040404050402115C9
:1000C000310541055105A1F70895F89484E0EFEE5C
:1000D000F0E0AEE6B0E0182E0E942F0FECE2F1E067
:1000E000A6E6B0E0182E0E942F0F91E0E9ECF0E0B8
:1000F000A4E6B0E0192E0E942F0FE2EEF0E0A3E993
:10010000B0E0182E0E942F0FEBEDF0E0AAE8B0E06F
:10011000192E0E942F0FE7EFF0E0A2E8B0E0182EB2
:100120000E942F0FEDE4F1E0A2E7B0E0182E0E944C
:100130002F0FE0E2F1E0A6E7B0E0182E0E942F0FAB
:10014000EEEDF0E0AAE7B0E0182E0E942F0FEBE1F1
:10015000F1E0AEE7B0E0182E0E942F0FE7E5F1E0E6
:10016000A6E8B0E0192E0E942F0FECE5F1E0AFE811
:10017000B0E0192E0E942F0FE3E5F1E0A7E9B0E00F
:10018000182E0E942F0FE3E0F1E0ABE9B0E0182E4B
:100190000E942F0FE0E1F1E0AFE9B0E0182E0E94DD
:1001A0002F0F7894089580E090E0A0E8BFE380935B
:1001B000EF009093F000A093F100B093F20080E084
:1001C00090E0A0E0B0E080932C0190932D01A093EB
:1001D0002E01B0932F0181E08093C9001092E200BC
:1001E0001092E3001092E4001092E5001092DB0000
:1001F000C49880E090E0A0EAB0E480934D01909331
:100200004E01A0934F01B093500180E090E0A0E236
:10021000B1E48093200190932101A0932201B09337
:10022000230180E090E0A0E7B1E48093DE009093AA
:10023000DF00A093E000B093E10080E090E0A0EA4E
:10024000B1E480931B0190931C01A0931D01B09316
:100250001E0183E08093570185E080935C0180E07C
:1002600090E0A8E4B2E48093530190935401A093EA
:100270005501B093560184EF91E0A0E0B0E0809387
:10028000030190930401A0930501B093060180E05F
:1002900090E0A0E0B0E48093100190931101A0934E
:1002A0001201B09313010E94650008951F920F92EE
:1002B0000FB60F9211242F923F924F925F926F923E
:1002C0007F928F929F92AF92BF92CF92DF92EF92E6
:1002D000FF920F931F932F933F934F935F936F93CF
:1002E0007F938F939F93AF93BF93EF93FF93CF939E
:1002F000DF93CDB7DEB72497DEBFCDBF8091580125
:1003000090915901A0915A01B0915B010097A1050C
:10031000B105A1F08091580190915901A0915A0125
:10032000B0915B010197A109B109809358019093A5
:100330005901A0935A01B0935B0101C0AF9860913D
:10034000EF007091F0008091F1009091F20020E0B8
:1003500030E040E050E00E94210E882309F476C08E
:100360006091FB007091FC008091FD009091FE0077
:100370002091E2003091E3004091E4005091E500CB
:10038000E0900301F0900401009105011091060135
:100390006090EF007090F0008090F1009090F2007B
:1003A00020901001309011014090120150901301E3
:1003B000A0902C01B0902D01C0902E01D0902F0163
:1003C000A982BA82CB82DC82621B730B840B950BF1
:1003D0000E94170E5B016C0117FD05C0C801B70133
:1003E0000E94170E14C0C801B70161707070807050
:1003F000907016950795F794E7946E297F29802BC6
:10040000912B0E94170E9B01AC010E94720D28E0F7
:1004100030E040E052E30E94910E20E030E04AE7F5
:1004200054E40E94910E9B01AC01C601B5010E94EB
:10043000910EA40193010E94910EA20191010E94CC
:10044000B40D29813A814B815C8169C06091FB00C8
:100450007091FC008091FD009091FE002091E200DF
:100460003091E3004091E4005091E500E0900301F9
:10047000F0900401009105011091060160901001B7
:1004800070901101809012019090130120902C0126
:1004900030902D0140902E0150902F01621B730B64
:1004A000840B950B0E94170E5B016C0117FD05C0B4
:1004B000C801B7010E94170E14C0C801B7016170CE
:1004C00070708070907016950795F794E7946E2978
:1004D0007F29802B912B0E94170E9B01AC010E945B
:1004E000720D28E030E040E052E30E94910E20E0DF
:1004F00030E04AE754E40E94910E9B01AC01C60132
:10050000B5010E94910E2AE038EE4CE151E40E94C0
:10051000B40DA40193010E94B40DA20191010E94A7
:10052000720D6093140170931501809316019093DE
:100530001701E0901401F09015010091160110913F
:10054000170160914D0170914E0180914F01909182
:1005500050012091E6003091E7004091E800509171
:10056000E9000E94720D9B01AC01C801B7010E9415
:10057000240E181684F460914D0170914E01809103
:100580004F019091500120E030E040E050E00E94A7
:10059000240E87FF32C0E0901401F0901501009105
:1005A00016011091170160914D0170914E018091DB
:1005B0004F01909150012091E6003091E700409169
:1005C000E8005091E9000E94710D9B01AC01C80147
:1005D000B7010E94210E88239CF460914D01709117
:1005E0004E0180914F019091500120E030E040E0B9
:1005F00050E00E94210E88231CF4D998AF9A66C05F
:10060000E0901401F090150100911601109117016E
:1006100060914D0170914E0180914F019091500178
:100620002091E6003091E7004091E8005091E90008
:100630000E94710D9B01AC01C801B7010E94210EFF
:10064000882384F460914D0170914E0180914F0197
:100650009091500120E030E040E050E00E94240EF4
:1006600087FF32C0E0901401F0901501009116014F
:100670001091170160914D0170914E0180914F01D1
:10068000909150012091E6003091E7004091E80000
:100690005091E9000E94720D9B01AC01C801B701A5
:1006A0000E94240E181694F460914D0170914E0131
:1006B00080914F019091500120E030E040E050E007
:1006C0000E94210E882314F4D99AAF98E090140167
:1006D000F090150100911601109117016091200111
:1006E0007091210180912201909123012091E600D7
:1006F0003091E7004091E8005091E9000E94720DAE
:100700009B01AC01C801B7010E94240E181684F4A5
:10071000609120017091210180912201909123012B
:1007200020E030E040E050E00E94240E87FF32C01D
:10073000E0901401F090150100911601109117013D
:1007400060912001709121018091220190912301FB
:100750002091E6003091E7004091E8005091E900D7
:100760000E94710D9B01AC01C801B7010E94210ECE
:1007700088239CF4609120017091210180912201D5
:100780009091230120E030E040E050E00E94210EF3
:1007900088231CF4D898AE9A66C0E0901401F090BB
:1007A00015010091160110911701609120017091BF
:1007B000210180912201909123012091E600309146
:1007C000E7004091E8005091E9000E94710D9B0103
:1007D000AC01C801B7010E94210E882384F4609106
:1007E000200170912101809122019091230120E04C
:1007F00030E040E050E00E94240E87FF32C0E090DD
:100800001401F090150100911601109117016091EB
:10081000200170912101809122019091230120916A
:10082000E6003091E7004091E8005091E9000E9415
:10083000720D9B01AC01C801B7010E94240E18166D
:1008400094F4609120017091210180912201909196
:10085000230120E030E040E050E00E94210E882398
:1008600014F4D89AAE98E0901401F090150100911C
:100870001601109117016091DE007091DF008091E8
:10088000E0009091E1002091E6003091E700409176
:10089000E8005091E9000E94720D9B01AC01C80173
:1008A000B7010E94240E181684F46091DE00709146
:1008B000DF008091E0009091E10020E030E040E036
:1008C00050E00E94240E87FF32C0E0901401F090A7
:1008D000150100911601109117016091DE007091D1
:1008E000DF008091E0009091E1002091E6003091DE
:1008F000E7004091E8005091E9000E94710D9B01D2
:10090000AC01C801B7010E94210E88239CF46091BC
:10091000DE007091DF008091E0009091E10020E026
:1009200030E040E050E00E94210E88231CF4C29881
:10093000AD9A66C0E0901401F09015010091160187
:10094000109117016091DE007091DF008091E0004E
:100950009091E1002091E6003091E7004091E8009D
:100960005091E9000E94710D9B01AC01C801B701D3
:100970000E94210E882384F46091DE007091DF00D4
:100980008091E0009091E10020E030E040E050E014
:100990000E94240E87FF32C0E0901401F0901501F0
:1009A00000911601109117016091DE007091DF0037
:1009B0008091E0009091E1002091E6003091E70005
:1009C0004091E8005091E9000E94720D9B01AC013A
:1009D000C801B7010E94240E181694F46091DE003D
:1009E0007091DF008091E0009091E10020E030E024
:1009F00040E050E00E94210E882314F4C29AAD9882
:100A0000E0901401F090150100911601109117016A
:100A100060911B0170911C0180911D0190911E013C
:100A20002091E6003091E7004091E8005091E90004
:100A30000E94720D9B01AC01C801B7010E94240EF7
:100A4000181684F460911B0170911C0180911D01A6
:100A500090911E0120E030E040E050E00E94240E22
:100A600087FF32C0E0901401F0901501009116014B
:100A70001091170160911B0170911C0180911D0163
:100A800090911E012091E6003091E7004091E8002E
:100A90005091E9000E94710D9B01AC01C801B701A2
:100AA0000E94210E88239CF460911B0170911C010F
:100AB00080911D0190911E0120E030E040E050E067
:100AC0000E94210E88231CF4C198AC9A66C0E09065
:100AD0001401F09015010091160110911701609119
:100AE0001B0170911C0180911D0190911E012091AC
:100AF000E6003091E7004091E8005091E9000E9443
:100B0000710D9B01AC01C801B7010E94210E882321
:100B100084F460911B0170911C0180911D019091E2
:100B20001E0120E030E040E050E00E94240E87FFEC
:100B300032C0E0901401F09015010091160110915F
:100B4000170160911B0170911C0180911D01909112
:100B50001E012091E6003091E7004091E80050919D
:100B6000E9000E94720D9B01AC01C801B7010E940F
:100B7000240E181694F460911B0170911C01809151
:100B80001D0190911E0120E030E040E050E00E9405
:100B9000210E882314F4C19AAC98609114017091CD
:100BA000150180911601909117012091EB00309171
:100BB000EC004091ED005091EE000E94210E882340
:100BC00084F48091140190911501A0911601B091C7
:100BD00017018093EB009093EC00A093ED00B0938D
:100BE000EE006091140170911501809116019091B1
:100BF00017012091F3003091F4004091F5005091DD
:100C0000F6000E94240E181684F48091140190912D
:100C10001501A0911601B09117018093F3009093F4
:100C2000F400A093F500B093F60060911401709168
:100C30001501809116019091170120915301309177
:100C4000540140915501509156010E94B40D20E08D
:100C500030E040E854E40E94910E0E94FA0D9B019E
:100C600044E0603074071CF02FEF33E005C0161627
:100C7000170614F020E030E039BD28BD789480914B
:100C80000F01882331F085E491E00E942F0A109231
:100C90000F012496F894DEBFCDBFDF91CF91FF9175
:100CA000EF91BF91AF919F918F917F916F915F91E4
:100CB0004F913F912F911F910F91FF90EF90DF90F7
:100CC000CF90BF90AF909F908F907F906F905F90EC
:100CD0004F903F902F900F900FBE0F901F90189540
:100CE0001F93CF93DF930E94140988E190E02FE0D7
:100CF0000FB6F894A89581BD0FBE21BDF894C3E648
:100D0000D0E0DE010E94160F802D8F3F39F40E9443
:100D1000D30080E0DE01082E0E94230F10921801FC
:100D200084E0EFEEF0E0AEE6B0E0182E0E941E0F79
:100D30006091EF007091F0008091F1009091F200CD
:100D400023EF3FEF47EC52E40E94240E181684F084
:100D50006091EF007091F0008091F1009091F200AD
:100D600020E030E040E050E00E94210E88237CF437
:100D700080E090E0A0E8BFE38093EF009093F00064
:100D8000A093F100B093F2008EE68093180184E006
:100D9000ECE2F1E0A6E6B0E0182E0E941E0F609192
:100DA0002C0170912D0180912E0190912F0120EF47
:100DB00033E244E759E40E94240E181684F060914F
:100DC0002C0170912D0180912E0190912F0120E82E
:100DD0003FE443EC57EC0E94210E88237CF480E032
:100DE00090E0A0E0B0E080932C0190932D01A093BF
:100DF0002E01B0932F0186E68093180121E0E9ECE3
:100E0000F0E0A4E6B0E0122E0E941E0F8091C9000F
:100E1000833028F02093C90084E68093180184E091
:100E2000E2EEF0E0A3E9B0E0182E0E941E0F8091E0
:100E3000E2009091E300A091E400B091E5008159B7
:100E4000904DA340B0405CF01092E2001092E3009D
:100E50001092E4001092E50083E980931801EBED15
:100E6000F0E0AAE8B0E0122E0E941E0F8091DB0095
:100E7000823030F01092DB008AE88093180104C0C1
:100E8000882311F0C49A01C0C49824E0E7EFF0E091
:100E9000A2E8B0E0122E0E941E0F8091F700909100
:100EA000F800A091F900B091FA0080549244AF404C
:100EB000B04078F084EF91E0A0E0B0E08093F700DC
:100EC0009093F800A093F900B093FA0082E8809321
:100ED0001801EDE4F1E0A2E7B0E0122E0E941E0F2F
:100EE00060914D0170914E0180914F0190915001A0
:100EF00020EF33E244E759E40E94240E181684F0F0
:100F000060914D0170914E0180914F01909150017F
:100F100020E83FE443EC57EC0E94210E88237CF448
:100F200080E090E0A0EAB0E480934D0190934E0100
:100F3000A0934F01B093500182E78093180184E0A1
:100F4000E0E2F1E0A6E7B0E0182E0E941E0F6091EB
:100F5000200170912101809122019091230120EFC5
:100F600033E244E759E40E94240E181684F060919D
:100F7000200170912101809122019091230120E8AC
:100F80003FE443EC57EC0E94210E88237CF480E080
:100F900090E0A0E2B1E48093200190932101A0931E
:100FA0002201B093230186E78093180184E0EEEDDF
:100FB000F0E0AAE7B0E0182E0E941E0F6091DE005C
:100FC0007091DF008091E0009091E10020EF33E22A
:100FD00044E759E40E94240E181684F06091DE0064
:100FE0007091DF008091E0009091E10020E83FE403
:100FF00043EC57EC0E94210E88237CF480E090E0C3
:10100000A0E7B1E48093DE009093DF00A093E000BE
:10101000B093E1008AE78093180184E0EBE1F1E00E
:10102000AEE7B0E0182E0E941E0F60911B01709178
:101030001C0180911D0190911E0120EF33E244E7D5
:1010400059E40E94240E181684F060911B017091DF
:101050001C0180911D0190911E0120E83FE443ECAA
:1010600057EC0E94210E88237CF480E090E0A0EAF7
:10107000B1E480931B0190931C01A0931D01B093D8
:101080001E018EE78093180191E0E7E5F1E0A6E804
:10109000B0E0192E0E941E0F80915701853030F06C
:1010A00083E08093570186E880931801ECE5F1E036
:1010B000AFE8B0E0192E0E941E0F80915C018A30CB
:1010C00030F085E080935C018FE88093180114E094
:1010D000E3E5F1E0A7E9B0E0112E0E941E0F609158
:1010E000530170915401809155019091560120EF68
:1010F00033E244E759E40E94240E18167CF480E0A1
:1011000090E0A8E4B2E48093530190935401A0933B
:101110005501B093560187E980931801E3E0F1E0AF
:10112000ABE9B0E0112E0E941E0F80910301909157
:101130000401A0910501B091060181569A4EA0408C
:10114000B04078F084EF91E0A0E0B0E0809303013C
:1011500090930401A0930501B09306018BE980935D
:101160001801E0E1F1E0AFE9B0E0112E0E941E0F9E
:101170006091100170911101809112019091130101
:1011800020E030E040EA51E40E94240E18167CF47E
:1011900080E090E0A0E0B0E4809310019093110112
:1011A000A0931201B09313018FE9809318017894F2
:1011B000C39880EA9FE00197F1F70E94DA0C85B5A9
:1011C0008F6085BD89B7806889BF8DE983BD0E9426
:1011D00049008AB383608ABB87B3866087BB84B3C8
:1011E000806F84BB20E030E0E0EAFFE0CF010197B0
:1011F000F1F72F5F3F4F24363105C1F78BB78F775B
:101200008BBF89B7806889BF20E030E0E0EAFFE06B
:10121000CF010197F1F72F5F3F4F24363105C1F71A
:101220008BB780688BBFFFCF80E189B988E98AB925
:1012300086E880BD10921F011092DD0008958AB1EA
:1012400087708AB908951F920F920FB60F921124DA
:101250008F939F93EF93FF939CB190936300809142
:101260006200843251F4993741F4809174008823EC
:10127000C1F481E08093740014C0809174008823CD
:1012800099F0E82FFF27EB5BFE4F90838F5F8093F1
:101290007400883049F481E080930F01109274004B
:1012A00003C080917400EDCF90936200FF91EF91A5
:1012B0009F918F910F900FBE0F901F9018951F92C6
:1012C0000F920FB60F9211248F939F93EF93FF937A
:1012D0009091DD0080911F01981781F0E0911F012E
:1012E000EF5FEF70E0936100E0931F01FF27EC597F
:1012F000FF4F8081809360008CB901C05598FF91A9
:10130000EF919F918F910F900FBE0F901F901895A6
:10131000282F9091DD009F5F9F7080911F0198178B
:10132000E1F3E92FFF27EC59FF4F20839093DD0075
:10133000559A08958FB7F8941092DD0010921F010E
:101340008FBF0895CF93DF93CDB7DEB724970FB645
:10135000F894DEBF0FBECDBFAC01DE011196FC01DB
:10136000838189839D012F5F3F4F8481FD018183AC
:10137000FA018581F9018183FA018681F90182836D
:1013800069817A818B819C8124960FB6F894DEBFA7
:101390000FBECDBFDF91CF910895CF93DF93CDB72F
:1013A000DEB724970FB6F894DEBF0FBECDBFAC01F9
:1013B000DE011196FC01838189839D012F5F3F4FE0
:1013C0008481FD018183FA018581F9018183FA011C
:1013D0008681F901828369817A818B819C8124963F
:1013E0000FB6F894DEBF0FBECDBFDF91CF91089549
:1013F0000F931F93CF93DF93CDB7DEB728970FB628
:10140000F894DEBF0FBECDBFFB0194E2998399E74C
:101410009A838B8330813C8341814D8392819E836B
:1014200023812F83380F940F930F290F28878E0164
:101430000F5F1F4FF80181918F010E948809CE0133
:10144000099608171907B1F728960FB6F894DEBF6A
:101450000FBECDBFDF91CF911F910F9108950F93D4
:101460001F93CF93DF93CDB7DEB724970FB6F894D1
:10147000DEBF0FBECDBFFC01DC01129620E092E082
:101480008D91280F9F5F9730D9F733813093750086
:101490008781281709F0D8C18F010E5F1F4F228165
:1014A0002093760027FFE8C0AF9B02C0AF9801C031
:1014B000AF9A8AE090E0A0E0B0E08093580190936A
:1014C0005901A0935A01B0935B01822F8F778093CB
:1014D0007600883009F4ACC08930A0F4843009F477
:1014E0004EC0853040F4823091F18330E0F5813098
:1014F00009F0C2C020C0863009F465C0873008F00A
:1015000086C055C08C3009F446C08D3038F48A301E
:1015100009F499C08B3008F09EC08DC08E3009F45C
:10152000A9C08E3008F4A3C0823109F458C08331B9
:1015300009F0A2C060C0CF010E94CD0960934D01A7
:1015400070934E0180934F019093500195C0CF014D
:101550000E94CD09609320017093210180932201A4
:101560009093230189C0CF010E94CD096093DE00D2
:101570007093DF008093E0009093E1007DC0CF0185
:101580000E94CD0960931B0170931C0180931D0183
:1015900090931E0171C0CF010E94CD096093E600B7
:1015A0007093E7008093E8009093E90065C0CF0155
:1015B0000E94CD0960932C0170932D0180932E0120
:1015C00090932F0159C0CF010E94CD096093EF0085
:1015D0007093F0008093F1009093F2004DC0CF0122
:1015E0000E94A20960930301709304018093050196
:1015F0009093060141C0CF010E94CD096093100174
:1016000070931101809312019093130135C0809162
:10161000FB009091FC00A091FD00B091FE00809332
:10162000E2009093E300A093E400B093E50024C0AF
:101630003093570121C03093DB00332311F0C49A5B
:101640001BC0C49819C030935C013A30A8F089E0FF
:1016500080935C0111C0CF010E94CD0960935301BA
:1016600070935401809355019093560105C00E94D8
:10167000D30002C00E946500F8012081209376000B
:1016800027FDEBC0822F8F50823008F0AF9A8AE09E
:1016900090E0A0E0B0E08093580190935901A093AE
:1016A0005A01B0935B01822F8F77809376008A3046
:1016B00009F4AEC08B30E0F4843009F461C08530A9
:1016C00050F4823009F454C0833008F055C08130A2
:1016D00009F0C3C049C0863009F47EC0863008F4E2
:1016E00077C0883009F484C0893009F0B6C088C05A
:1016F000803109F44DC0813150F48C3009F444C07C
:101700008C3008F48DC08F3009F0A7C00FC0833132
:1017100009F46AC0843120F4823109F09EC060C0AF
:10172000843139F08E3709F098C07EC064E171E0F1
:1017300017C060911401709115018091160190916C
:10174000170120E030E04AE754E40E94910E0E9425
:10175000FA0D69837A838B839C83BE016F5F7F4F11
:101760008FE00E94F80979C06DE471E081E0F9CF63
:1017700060E271E082E0F5CF6EED70E083E0F1CFE2
:101780006BE171E084E0EDCF66EE70E08CE0E9CFD4
:1017900010927500D99903C081E080937500D899A3
:1017A00005C080917500826080937500C29905C064
:1017B00080917500846080937500C19905C0809107
:1017C000750088608093750065E770E080E1C9CF9F
:1017D0006CE271E085E0C5CF6FEE70E086E0C1CFCE
:1017E00063E071E082E1BDCF60E171E083E1B9CFF8
:1017F000809157018093750065E770E088E0B1CF74
:101800008091DB008093750065E770E089E0A9CFE7
:1018100080915C018093750065E770E08AE0A1CF5C
:1018200063E571E08BE09DCF8EEA97E4A1E8BFE32A
:101830008093400190934101A0934201B0934301F2
:1018400060E471E08EE78DCF8091190190911A01CB
:10185000019690931A018093190124960FB6F8947B
:10186000DEBF0FBECDBFDF91CF911F910F910895C5
:101870001F920F920FB60F921124EF92FF920F93C7
:101880001F932F933F934F935F936F937F938F9308
:101890009F93AF93BF93EF93FF93109277001092B3
:1018A00078001092790010927A0085E0982F9A952E
:1018B000F1F7C69A8A95F1F7839B0CC080E090E01F
:1018C000A0E8BFEF8093770090937800A093790011
:1018D000B0937A00C69887E180937B0020917700CF
:1018E000309178004091790050917A00E6E1F0E083
:1018F00065E091E0E92EF12C012D112D862F8A95BE
:10190000F1F7C69A862F8A95F1F7839B0EC0D8010E
:10191000C7010E2E04C0880F991FAA1FBB1F0A946F
:10192000D2F7282B392B4A2B5B2BC69831978FEF98
:10193000EF3FF80719F72093770030937800409332
:10194000790050937A0010927B00862F8A95F1F7E8
:10195000C69A6A95F1F7C6981092440184E05595AD
:101960004795379527958A95D1F7CA01B9010E9405
:10197000F50C6093FB007093FC008093FD00909346
:10198000FE00A8958AB780628ABFFF91EF91BF9150
:10199000AF919F918F917F916F915F914F913F9107
:1019A0002F911F910F91FF90EF900F900FBE0F900E
:1019B0001F901895BB9ABC9ABD9ABE9A8B98C598F1
:1019C000C69880E49CE9FC013197F1F7C59AFC01C7
:1019D0003197F1F7C5980197F1F78AB780688ABF08
:1019E0008BB780688BBFC59A0895AF92BF92CF9294
:1019F000DF92EF92FF920F931F93CF93DF93AB0190
:101A0000BC0110927D0010927E0010927F00109217
:101A1000800010927C00C0905C01CC2DDD272197C6
:101A2000EE24FF248701DD241FC05F01AA0CBB1C2C
:101A3000AA0CBB1C95012B553F4FF9018481958160
:101A4000A681B78180839183A283B38321E830E0AC
:101A5000A20EB31EF50180839183A283B383E80EA7
:101A6000F91E0A1F1B1FD394ED2DFF27EC17FD074E
:101A7000E4F2E0927D00F0927E0000937F001093EC
:101A80008000D0927C00FE01EE0FFF1FEE0FFF1FC3
:101A9000DF01AB55BF4F4D935D936D937C931397CF
:101AA000EF57FF4F4083518362837383F1E0FC154E
:101AB00058F49E01442737FD4095542FC801B701C3
:101AC0000E94D90EBA01A901CB01BA01DF91CF91D1
:101AD0001F910F91FF90EF90DF90CF90BF90AF904C
:101AE00008955058192EEFD001D0D2C0BA1762070E
:101AF000730784079507B1F188F40EF410940B2E48
:101B0000BA2FA02D062E622F202D072E732F302DD9
:101B1000082E842F402D092E952F502DFF27552359
:101B2000B9F0591B49F0573E98F0469537952795DF
:101B3000A795F0405395C9F776F0BA0F621F731F4F
:101B4000841F30F4879577956795B795F040939506
:101B500017FA0F2E0895BF1BBB27BA0B620B730B2E
:101B6000840BF6CFDEF6DBC0AED001D091C055239A
:101B700059F0992369F09F575F57951B33F442F44E
:101B8000903811F4915805C09BC091589F3F09F4BB
:101B9000C6C0BB27112462177307840730F4660F91
:101BA000771F881FBB1F915098F311D00F920FD051
:101BB0000F920DD0A0E82617370748071B0609F03B
:101BC000A048BA2F602D7F918F9100240895A0E83E
:101BD0000024621773078407B10528F0621B730B9A
:101BE000840BB1090A2A660F771F881FBB1FA695B1
:101BF00081F7089597FB73D09F3738F0FEE9F91B02
:101C0000982F872F762F6B2F05C086C096958795C6
:101C100077956795F150D0F73EF490958095709543
:101C200061957F4F8F4F9F4F0895E89403C097FBB6
:101C30000EF4F3DFB62F672F782F892F9EE900244B
:101C400027C00ED05EF004C00BD026F001C008D033
:101C500019F020F48FEF089580E0089581E0089551
:101C600097FB092E052600F8689430D0E89407FC0D
:101C700007C0621773078407950721F008F40094E2
:101C80000794989408959A95BB0F661F771F881F35
:101C900011249923A1F08823B2F79F3F59F0BB0F7D
:101CA00048F421F4002011F460FF04C06F5F7F4FFF
:101CB0008F4F9F4F881F9795879597F908952CC050
:101CC0009FEF80EC0895052E092607FA440F551F53
:101CD0005F3F79F0AA27A51708F051E04795880FD4
:101CE000991F9F3F31F0BB27B91708F091E0879506
:101CF00008959F919F911124E3CF97FB880F991F1F
:101D00009F3F31F0BB27B91708F091E08795089500
:101D10009F919F911124D4CF6627772788279927F1
:101D20000895D1DF01D0B4CF992339F0552329F09C
:101D30009F575F57950F13F49AF1F1CF91589F3F3A
:101D4000E1F3629FA12D0F92BB27639FA00DB11DF0
:101D5000EE27729FA00DB11DEE1FAF93AA27649FBF
:101D6000B00DE11D739FB00DE11DAA1F6627829F74
:101D7000B00DE11DA61F5527749FE00DA11D551F35
:101D8000839FE00DA11D561F849FA00D511D852F1F
:101D90007A2F6E2F1F900F9088231AF4939539F4A1
:101DA0008FCF000C111CBB1F661F771F881F0128D7
:101DB000089597FB092E05260ED057FD04D014D0A8
:101DC0000AD0001C38F450954095309521953F4F2E
:101DD0004F4F5F4F0895F6F79095809570956195F8
:101DE0007F4F8F4F9F4F0895A1E21A2EAA1BBB1B56
:101DF000FD010DC0AA1FBB1FEE1FFF1FA217B307D7
:101E0000E407F50720F0A21BB30BE40BF50B661FEC
:101E1000771F881F991F1A9469F7609570958095B0
:101E200090959B01AC01BD01CF010895E199FECFD2
:101E3000BFBBAEBBE09A11960DB20895F7DF0192D9
:101E40001A94E1F70895E199FECFBFBBAEBB0DBA7E
:101E500011960FB6F894E29AE19A0FBE0895019098
:0A1E6000F2DF1A94E1F70895FFCFB6
:00000001FF
